:1000000000308A00A82800000030A1001F08C33972
:1000100021049F000D30A000A00B0C289F149F18F6
:100020000F281E08A601A500260CA300250CA2007F
:10003000A30CA20CA30CA20CA30CA20C2208AB00D4
:100040000430A1001F08C33921049F000D30A00017
:10005000A00B28289F149F182B281E08A801A70072
:10006000280CA300270CA200A30CA20CA30CA20C2A
:10007000A30CA20C2208AC000C30A1001F08C3394D
:1000800021049F000D30A000A00B44289F149F184E
:1000900047281E08AA01A900003447308400000840
:1000A00003195F280230A100A001A00B5528A10B65
:1000B00054289730A000A00B5B28800B52280034F6
:1000C0000830C802031C6F28483084000310800CDD
:1000D000000803196F286D280000800B6C2800347D
:1000E000C7014708293C031C842805150830A000D7
:1000F000A00B7828000005110330A000A00B7E287B
:1001000000000000C70A71280330C700C630C800CD
:100110006020C70B8628DC29C7014708143C031C54
:10012000A02805150830A000A00B94280000051198
:100130000330A000A00B9A2800000000C70A8D28F9
:100140000330C700C630C8006020C70BA228DE29D4
:1001500084011F3083051F1383161F149F141F155E
:100160009F15073083129F00703083168F001B305D
:10017000650083121F1383161F149F141F119F15F0
:100180001F129F161F1383129F131F1470308316A4
:100190008F00831285120420A608031DD32825088A
:1001A0000C3C0318D728AF010330B000DB28013026
:1001B000AF000230B000A608031DE2282508023C6B
:1001C0000318E4280420DB28AD0130082D020318B1
:1001D000F3288516FA30C7004D208512FA30C70083
:1001E0004D20AD0AE5280130B200B301B401B500DD
:1001F000B600C6010420051185122F0B0229B70194
:10020000B8010829AF08031D0829B7010130B8005B
:100210002B080F3C031D0E290E30AB00AD012D083D
:10022000033C031C2B290F30AB052B08B100013018
:10023000B105310B22292D080A3C323E84000130E1
:10024000800027292D080A3C323E840080010310DB
:10025000AB0CAD0A0F29851D3A290B30AD002D08D6
:100260000E3C031C392932302D0784008001AD0A71
:100270002F2960292C08053C031C4D290B30AD00AB
:100280002D080E3C031C4C2932302D078400013010
:1002900080008516AD0A402960292C08093C031806
:1002A00060290B30AD002D080D3C031C5E29323057
:1002B0002D07840080018516AD0A53290130C00046
:1002C0002C08063C031C7E290130C1002C08023C8E
:1002D000031C6E29C2010130C3007D292C08043C97
:1002E000031C76290130C200C3017D292C08063C7D
:1002F000031C7D290130C200C3009929C1012C08CB
:10030000083C031C8629C201C30199292C080A3C18
:10031000031C8E29C2010130C30099292C080C3C12
:10032000031C96290130C200C30199290130C20083
:10033000C300AE010330AD002D080F3C031CAF29F4
:1003400032302D0784000310000DAE0701302D0759
:10035000323E84000008AE070230AD079C29430BF3
:10036000B4290310430DAE070330AE05AE08031DDC
:10037000BD290130C400C500D1292E0BC329C401F9
:100380000130C500D1292E08023C031DCB290130C4
:10039000C400C501D1292E08033C031DD129C40185
:1003A000C501AD012D08143C031CE02932302D0796
:1003B0008400000BDD297028DE298C28AD0AD229A3
:1003C0000511AA08031DE9292908DB3C031CE929BA
:0C03D0008516DC30C7004D20F3286300C8
:02400E00C43FAD
:00000001FF
